:030000000219FDE5
:03000B000200A848
:03002B000201636C
:03005B000202EDB1
:030073000202D3B3
:1000800002030406080C10182030406080040608A3
:100090000C10182030406080A0C000070F1F3F05E3
:1000A000050D050305030302C2AFC0D0C0E0206206
:1000B00017E5256002E473E525F4F58A758B00D217
:1000C00062D0E0D0D0D2AF3285268AC262E526F473
:1000D0006035306803207210758B00D0E0D0D0C23C
:1000E00093C295C297D2AF32C293C295C297206E87
:1000F0000C206609740AD5E0FDE57E4290758B0000
:10010000D0E0D0D0D2AF32758A00C28DD26201FD6C
:1001100001B7306805206602D29301B73068052028
:100120006602D29501B7306805206602D29701B702
:10013000C29230680A2066077408D5E0FDD29301A8
:10014000B7C29430680A2066077408D5E0FDD295DE
:1001500001B7C29630680A2066077408D5E0FDD260
:100160009701B7C2AFC2AD53E6EFC0D0C0E0D2D363
:10017000D2AFC2CEE52A6007207449152A21C4787F
:1001800000790020742EE580307E01F430E302789F
:10019000FF53DACF207E0343DA20307E0343DA10A8
:1001A000C2D8C271E580307E01F430E30279FFC32A
:1001B000E89970CB306103752A18207403752A18EA
:1001C000885FD27020740DE52B6004152B21D44379
:1001D000DA01C2D82070024136A85F206102C270E5
:1001E000207431C3E894F0400374F0F8E8C4540F6D
:1001F00028F87984B703024114C313C3138721205D
:100200000802C313200A06C3C898F8411428F850FE
:100210000374FFF8C3E895685003E568F88822E5A1
:100220002D54066011E533C313C31324062522F5AC
:100230002250037522FF852224A824C3E524956457
:100240004002A8648825E5697002417AC3E8AA697A
:100250009A5003E8FAE4F9EAC333FBE56BF45B294F
:10026000400D256AF8E56A6002156A400B417A0A7A
:10027000C3E56A9A5002056A78FF8826C26EC3E514
:100280002694F84002D26EC3E52594404002D26421
:1002900020CF0AD0E0D0D043E610D2AD32C2CF0595
:1002A0003A7801E52A6005307402152AC3E55F94A7
:1002B00001400575620041C9756300756C00E56217
:1002C0002401F56250037562FFD0E0D0D043E61000
:1002D000D2AD32C2AFC0D053E67FC2607591008507
:1002E0005694855795759104D0D0D2AF32C2AF5392
:1002F000E6EFC2ADC0D0C0E0C0F0D2D3D2AFA8FB11
:10030000A9FCC2D8307102615453DACF207E034376
:10031000DA10307E0343DA20D271E580307E01F4BA
:1003200020E302612B88278928A18153DACF207E20
:100330000343DA20307E0343DA10C2D8C27130742E
:1003400002A16D7800E580307E01F430E302A16DFA
:10035000885FA15553DACF207E0343DA20307E0335
:1003600043DA10C271206102812D53DACF207E035F
:1003700043DA10307E0343DA20C2D8D271885A891A
:100380005BC3E89558F8E99559F97B007E087A0037
:10039000C3E8948CE994005005755E00811F8821A4
:1003A00078A2E6A8216055C3E894C8E994005008F3
:1003B000E4D2E4FB7A0A61FAC3E89468E994015054
:1003C00008E4D2E3FB7A0F61FAC3E894D0E994021F
:1003D0005008E4D2E2FB7A1E61FAC3E894A0E994E3
:1003E000055008E4D2E1FB7A3C61FAC3E89498E94D
:1003F00094085008E4D2E0FB7A787E00C3E8955C6C
:10040000FCE9955DFD30E70AECF42401FCEDF434E1
:1004100000FD755E00C3EC9AED9E5003755E018889
:100420005C895D855A58855B597802A155C3E8956A
:1004300027F8E99528F9307C02A139307B02A139EF
:10044000307A02A1322075028150E9FDE8FC816F0B
:10045000E9C313F9E813F8307902A132E9C313F9BB
:10046000E813F8307802A132E9C313FDE813FC2049
:0E047000612CC3EC941CED940240028186EDD9
:10047E00701EC3EC94C850180529E5297002152981
:10048E00C3E529940A5002A16D755F00D270A16D6B
:10049E00E529600215297888E6F97400207F08782E
:1004AE0096B90302789EE624FAFEE43400FFC3EC0C
:1004BE009EFCED9FFD9208B90310A208500720760E
:1004CE0009D27681D8307602C276A2085016B903C8
:1004DE000DECF42401FCEDF43400FD0204F278007E
:1004EE007900A139B90315EC33FCED33FDC3EC945F
:1004FE000AFCED9400FD50047C007D00C3EC94FFDB
:10050E00ED9400400678FF7900A139EC8575F0A4D2
:10051E00C5F0A2F733F87900400302055578FF794C
:10052E0000020555E9C313F9E813F8307C0EE960B3
:10053E000278FFC3E81338F8E43400F9C3E894FFF7
:10054E00E99400400278FF885FD270206102A16DAD
:10055E00741FF4552F4BF52FC274EB7002D27475C5
:10056E002A18307403752A0A306102A1812074039F
:10057E0053DAFE207403752B06D0F0D0E0D0D0D223
:10058E00AD43E6103279010205B179030205B17966
:10059E000A0205B1791E0205B179640205B179C866
:1005AE000205B17817E4D5E0FDD8FAD9F6227A140F
:1005BE007B780205D87A107B8C0205D87A0D7BB435
:1005CE000205D87A0B7BC80205D87902B27DE4C247
:1005DE0094D5E0FDD295D5E0FDC295D5E0FDD2943F
:1005EE00D5E0FDD293E576D5E0FDC2937496D5E0C5
:1005FE00FDD9D9EAF8D5E0FDD8FBDBCEC29422C3F3
:10060E007C007D0075F00005F0EA33FAEB33FB5009
:10061E00F6EB13FBEA13FAC3E9FFE8FEE89AF8E9F2
:10062E009BF95004EFF9EEF8B3EC33FCED33FDD546
:10063E00F0DFEDF9ECF822E889F08A20D2D4F8A99F
:10064E00F07B0030F70B7BFFF42401F8E9F4340063
:10065E00F9E88520F0A4ADF0F8E98520F0A4AFF01C
:10066E00FEED2EF974003FFA7C04C3EA13FAE91387
:10067E00F9E813F8DCF48BF030F70AE8F42401F80B
:10068E00E9F43400F9E889F0C2D4F8A9F02222C3C3
:10069E00E54113F9E54013F8C3E54598F8E54699A9
:1006AE00F9500CC3E89480E994FF40160206D4C3B7
:1006BE00E8947FE9940050030206D4787F79000213
:1006CE0006D4788079FF884A894B22E54A2547F877
:1006DE00E54B3548F9854B20E4300701F43549FAEE
:1006EE0030E709C3EA94F04015020712C3EA940FEB
:1006FE00500302071278FF79FF7A0F020712780073
:10070E0079007AF0C3E5249564500AC374019524E8
:10071E00500B020730E54B20E70E020730E54B3059
:10072E00E706884789488A492278A4E6FAC3E54A4B
:10073E0033F8E54B33F9D145E930E70BC3E8948044
:10074E00E994FF4013E16AC3E8947FE994005002F4
:10075E00E16A787F7900E16A788079FFE820E71511
:10076E00C3E52398F84009C3E894014003020791BA
:10077E007801020791E8F424012523F840030207CB
:10078E009178FF884C2278A5E6FAA848A949D14568
:10079E00E930E70CC3E89401E994FF40160207C55F
:1007AE00C3E894FFE9940050030207C578FF79006F
:1007BE000207C5780179FFE920E715C3E54C98F8E3
:1007CE004009C3E8940140030207EC78010207ECEC
:1007DE00E8F42401254CF840030207EC78FF882446
:1007EE002278FFC26420693D206A12D264C3E541BB
:1007FE00940A4009C3E52594405002C26479A1E7EA
:10080E006023E541601F74FF8541F0848539F03027
:10081E006A0375F005A4F8C5F0600278FFC3E89589
:10082E00675002A867886622C3E5409440E541946C
:10083E0001E5665003140147046002F566220208C2
:10084E004F2275E890227883E6FFE5E820ECF7A8C2
:10085E00BDA9BE0573C3E57394084052757300E9D4
:0D086E00FA79A0E76044EA7007E574601BAA
:10087B0002088AC3E895746010E5745006600C1486
:10088B000208960460F9020896E574F574C394A8FF
:10089B00401B7564C0C394054013756480C39405F5
:1008AB00400B756440C39405400375640075BB0130
:1008BB0022E564F460020564E573B4070375BB1E9F
:1008CB0022743279A687F0A4C5F0A2F733F8C3E8F7
:1008DB0095644002A8648822882488258826886726
:1008EB00227540007541F022C2AF75C820A8CCA973
:1008FB00CDAA3A30CF010A75C824D2AFAB3BAC3C82
:10090B00883B893CC3E89BF8E99C206908F9306770
:10091B000241082165AD3D8A3DF9EA9DFA600478F4
:10092B00FF79FFAE3EAF3F8B3E8C3FC3EC9FFCC3CA
:10093B00E99CF542A83BA93CC3E89EF8E99FF9C3A3
:10094B00E54113FBE54013FAE82AF540E93BF54195
:10095B0050067540FF7541FF21AFAA40AB41AC403B
:10096B00AD417E047F02C3EB940440021E1FC3EB18
:10097B00940840021E1FC3ED13FDEC13FCDEF7C3FE
:10098B00EA9CFAEB9DFBEF6009C3E913F9E813F856
:10099B00DFF7EA28FAEB39FB8A408B4150067BFFE5
:1009AB008B408B41C3EB94025002D2673069047FBA
:1009BB000321DA7892E6FFC3E537948240110FC327
:1009CB00E53794A040010FC3EF940640027F057EEC
:1009DB0005E541C4540FF9E541C454F0F8E540C4B2
:1009EB00540F28F8C3E89EFAE99400FB4009C3EAC8
:1009FB009402EB940050047A02E4FB4154AA40ABFE
:100A0B0041EBC4FEEAC4540F4EFCC3EA9CFAEB94D0
:100A1B0000FBC3E813C313F8EA28FAEB3400FB8A94
:100A2B00408B41C3EB94024002C2677805EBC4FED6
:100A3B007B00EAC4540F4EFAC3EA98FA4005C394FC
:100A4B000250027A027892E6FF30600241548552DE
:100A5B0056855357D26043E680C3E49AF8E49BF97A
:100A6B0030670241EEE8FAE9FBD3E913FDE813FC2A
:100A7B0088528953C3EF94036038EF20E00DE82CC4
:100A8B00F8E93DF9ECFAEDFB020AA9E828F8E93997
:100A9B00F9C3E82402F8E93400F97AFE7BFFC3EFCF
:100AAB009403400E8A548B55884E894F8C508D5130
:100ABB006122885489558A4E8B4F8C508D513069E9
:100ACB0020C3E53394034019E542A2E713F8E5553B
:100ADB00F4240138400B20E7087554FFF42401F58A
:100AEB00556122E8FAD3E813FC8852C3EF940360F4
:100AFB0020EF20E007E82CF8ECFA610EE82824023E
:100B0B00F87AFEC3EF940340088A54884E8C5061E8
:100B1B002288548A4E8C50E56BC3335002646BF5BC
:100B2B006B306002612C753402D26043E680E52D98
:100B3B0054066026A840A941C3E913F9E813F8C28B
:100B4B00AF53E67F759100C3E498F594E499F5955E
:100B5B00759104D26043E680D2AF22D26575440012
:100B6B00752000306B03752040020B85D2657544F0
:100B7B0000752040306B03752000D2AF78012067E1
:100B8B0022E52D54066002C265C3E541940540136E
:100B9B007802940540087803940540027806306982
:100BAB0002780A206019E544601530690AC3E53301
:100BBB0094034003D53406D2AFD26C815F7134D22B
:100BCB00AF0000C2AF206726E541C3FB940F400284
:100BDB007B0FEB240530730123306A0274282062EB
:100BEB000123F93069027982E58BC39940B505443D
:100BFB00E59E7005E59B020C06E59A5440B5200274
:100C0B00814930690A08C3E8940A40010861AE20A3
:100C1B0065026185C26553E67F759100306710757B
:100C2B0094007595FE759104D26043E6806185AEA4
:100C3B0040AF41C3E49EF594E49FF5958130C3E545
:100C4B00339402500261853065026185D802815D63
:100C5B0061AEC26C53E67F759100855494855595B2
:0E0C6B00759104854E56854F57D26043E68042
:100C7900D2AFE52D54066008206A020533020C99AB
:100C8900306C0D206B0A2065071581158102153F0F
:100C99002278003064053065027801E53775F00780
:100CA900A4F9E5F028F5F0E9A2F013A2F113A2F2F4
:100CB90013F537C394785003753778C3E5379538FA
:100CC9004008D266C293C295C29730600281D3852B
:100CD9005056855157D26043E68022207D14C2AF19
:100CE900754302C294D292D2AF759F33759E0002AA
:100CF9000EC5C2AF754302C294D296D2AF759F3367
:100D0900759E00020EC5307243207D20C2AF754327
:100D190003900141757E10C297C296306204D29544
:100D2900A12DD294D2AF759E23020EC5C2AF7543D1
:100D390003900141757E10C293C292306204D2952C
:100D4900A14DD294D2AF759E22020EC5207D17C245
:100D5900AF75430390011CC297306202D295D2AF9E
:100D6900759E23020EC5C2AF75430390011CC29341
:100D7900306202D295D2AF759E22020EC5207D1136
:100D8900C2AF754304C292D296D2AF759E22020EAB
:100D9900C5C2AF754304C296D292D2AF759E2302E3
:100DA9000EC5307249207D23C2AF754305900130CD
:100DB900757E04C295C294306204D293A1C9D292BD
:100DC900D2AF759F33759E00020EC5C2AF7543053C
:100DD900900152757E40C295C294306204D297A1A7
:100DE900ECD296D2AF759F33759E00020EC5207D59
:100DF9001AC2AF754305900112C295306202D293AF
:100E0900D2AF759F33759E00020EC5C2AF754305FB
:100E1900900126C2953062E8D297D2AF759F33759B
:100E29009E00020EC5207D11C2AF754306C296D23F
:100E390094D2AF759E23020EC5C2AF754306C29206
:100E4900D294D2AF759E22020EC5307242207D2007
:100E5900C2AF754301900152757E40C293C2923070
:100E69006204D297C171D296D2AF759E22020EC585
:100E7900C2AF754301900130757E04C297C29630A6
:100E89006204D293C191D292D2AF759E23C1C5207B
:100E99007D16C2AF754301900126C293306202D21A
:100EA90097D2AF759E22C1C5C2AF75430190011299
:100EB900C297306202D293D2AF759E23C266229046
:100EC9000110757E00C293C295C297C292C294C2A4
:100ED90096C26222788076FF0876FF0876FF087648
:100EE900FF08760308760408760708760308760172
:100EF900087601788C76010876FF0876FF0876FF78
:100F09000876FF0876FF0876030876FF0876FF085B
:100F190076FF0876250876D00876FA0876FA0876F4
:100F2900040876FF08760108760008767A0876FFC5
:100F3900087601087601087600087603227887E6A4
:100F4900FFC272BF0302D2727888E6C394036008B5
:100F5900C27DE630E102D27DC27E7889E630E102C7
:100F6900D27EC3EF94026008758E01D273020F7EA0
:100F7900758E00C273227880E6149000809378A45D
:100F8900F67881E6149000809378A5F67886E614C1
:100F990090008D9378A6F6789CE67538FF75390C24
:100FA900B402067538A075390AB403067538827516
:100FB900390578A3E61490009A93F569D1C82222DD
:100FC9007896E6FA7897E6FB7888E6B40305C3EBEA
:100FD900940EFB307F047A007BFFC3EB9AFCC39429
:100FE9008250027C827575000575EC8575F0A4C385
:100FF900E5F0947D40F222D27F120FC91205A27A40
:10100900007B007C10120598E55F2AFA74003BFB0F
:10101900DCF37C04C3EB13FBEA13FADCF7FEC27FB3
:10102900120FC922E5EF20E6037520000520903D47
:10103900FFE520146006901FFF146000930460030D
:1010490075EF1253D9BF7581C043FF80120593759F
:10105900EF0243B203E5B3240420E70DF521E5B11E
:0F10690020E0068521B343B101120EC87580083F
:1010780075A40075F1FF75D4F775900275A5FC7518
:10108800F2FC75D50075A0FD75A60275F30275D63C
:101098000075B0FF75A70175F4FF75E241E4F8F635
:1010A800D8FD756B01120EDD12158178988676755C
:1010B8003001C2AF1205AC1205BC1205A21205C35D
:1010C8001205A21205CA1205A212169A1205AC122E
:1010D80005AC1205A7C2AF78FA79FA308307D9FBB5
:1010E800D8F7021C00120F46120F7F120FC8120FFA
:1010F800C978988676120EC875885075891275C891
:101108002475910475D84075A82275B80275E690C3
:10111800759B80759D00759A80759C0075D10E75BC
:10112800BC5875BB0175BA1F75E880120593D2AF1C
:1011380012084C53DACF207E0343DA20307E034373
:10114800DA1043DA01C2D8C2711205ACD2617B034E
:101158007A0CE55E70077A0CDB030210DD1205A23B
:101168002070030210DDC270E55FC3940240E1E520
:101178002F541F856160F561B560D5DAD5C261531A
:10118800DACF207E0343DA20307E0343DA10C2D858
:10119800C27178A2E67008D274E52F54E0F52FC228
:1011A800757529001205A7307409C3E529940A400A
:1011B80002D27512059878023074027800C3E55F90
:1011C8009840F0C2AF1205BC1205BC1205BCD2AFE4
:1011D8001205AC754D007888E6B4030241C11205CA
:1011E80098788CE6C3940150030212C1E530C39489
:1011F8000150030212C1207435C3E55F94FF500308
:101208000212C1C2AF1205D1D2AF1205A7C3E55F62
:10121800940150EFC2AF1205BC12059D1205BCD255
:10122800AF1205A7C3E55F94FF40E902171F7F05CA
:10123800D27F120FC91205A7C2AFC27F120FC9AE63
:101248005FC3E55F947FD2AF4079120593C2AF12B6
:1012580005D1D2AFDFDA1100C3EE94057897F61204
:1012680005AC1215C31216A27F0AD27F120FC9123B
:1012780005A7C2AFC27F120FC9AE5FC3E55F947FF7
:10128800D2AF50E4120593C2AF1205BC12059D12ED
:1012980005BCD2AFDFD41100EE24057896F612050E
:1012A800AC1215C31216D11205A7120FC9C3E55FF8
:1012B80094FF500221FE02171FC3E55F954D4003BE
:1012C800855F4D1205A778017988E7B40302780590
:1012D800C3E55F98400221DEC2AF1205D11205D1E5
:1012E8001205D1D2AF1205AC753000E4F531F532F4
:1012F8000531E531F470390532789AE678191460C9
:1013080012783214600D787D14600878FA1460033E
:10131800753200C3E53298401715327531B47899A3
:101328008676C2AF1205D1D2AF789886761205A715
:1013380012059DE52A700530740201DD78012074DC
:10134800027806C3E55F9840A77888E6C3940360EF
:10135800031205A7E52A70030210DDC2AF120EC8FA
:10136800E4F522F523F524F525F526F56AD2AF78BC
:1013780085E6C333F568E4F545F546F547F548F5E0
:1013880049F573F52CF52DF53775730875BB1E12E5
:101398000593120850E5E820ECFBA8BDA9BEE9704A
:1013A80001F8887412085475730875BB1E7887E6AF
:1013B800FE7602120F467887EEF6C2AF7564FF120A
:1013C80008CC852264852265852266D2AF75220104
:1013D80075240175250175260185636C756D017885
:1013E80088E6B40307C27D307602D27DD268D2691E
:1013F800753300120E2E120E531208EC1208F31257
:1014080008EC1208F31208EC021420C2AF120F46BF
:10141800D2AF75730075BB01120B7712069C120CC4
:101428009A120CE41208F3120B66306D0312069D33
:101438002067031207EF306703120836120C9A125E
:101448000D0F1208F3120B77306D031206D9120C28
:101458009A120D861208F3120B66306D03120737C5
:0F146800120C9A120DAB1208F3120B77306D03B2
:10147700120794120C9A120E2E1208F31208501229
:101487000B66120C9A120E531208541208F33069A5
:1014970032206B2F85676485676585636C756D0181
:1014A70079187A0CC3E53399400CC269D26A8A3538
:1014B7007564FF0214CAC3E55F9401400302142058
:1014C700021547306A1B206B18E535147004C26A91
:1014D7008113F535C3E55F9401400302142002151B
:1014E70047753600C3E5627882985054307404E536
:1014F7002A604D7888E6B40317207D05207607A17A
:1015070017307602A117206B07D26B856764815F5E
:1015170078F0306B058567647820C3E54198500201
:101527008120306B1BC26BC27D307602D27DD26ABE
:1015370075351285676481200536E55F6002A14A2B
:10154700753600C2AF120EC87887E6FE7602120F14
:10155700467887EEF6E4F522F523F524F525F526FA
:10156700F568C268D2AF120593120EC8307409C36A
:10157700E5369405400201DD41F3901A0D782012FB
:101587001605E520B45A0CA3121605E520B4A503E9
:101597000215A3120EDD1215C30215C2901A0378A5
:1015A700807B0A121605A308DBF9901A0F788C7B4B
:1015B70018121605A308DBF9901A2722C2AF1216D4
:1015C7004412161E901A00740E12160AA3740412FF
:1015D700160AA3741412160A901A0378807B0A124B
:1015E7001609A308DBF9901A0F788C7B18121609D5
:1015F700A308DBF9121657121635901A2722E4931F
:10160700F622E6438F01538FFD75EF0275B7A57577
:10161700B7F1F0538FFE22438F02438F0175EF021C
:1016270075B7A575B7F1901A0DF0538FFC22901A74
:101637000D745AD10A901A0E74A5D10A227A3079FC
:10164700D07820901A40D105E520F709A3DAF722D0
:101657007A3079D0901A40E7D10A09A3DAF922AB98
:1016670077A878BB01027984BB02027985BB0302A4
:101677007986BB04027992BB05027987BB0602799A
:10168700A3BB0702799CBB08027988BB0902798949
:10169700E8F7227C051205ACDCFB22C2AF1205BCC1
:1016A7001205C31205CA1205D112059D1205BC12F7
:1016B70005C31205CA1205D112059D1205BC1205F4
:1016C700C31205CA1205D1D2AF22C2AF1205D11279
:1016D70005CA1205C31205BC12059D1205D11205D4
:1016E700CA1205C31205BC12059D1205D11205CAFF
:1016F7001205C31205BCD2AF22AE77AF78C2AF12C4
:1017070005BC1205BC1205BC12059DDEF21205D1FF
:1017170012059DDFF8D2AF22D1A2D19AD19A75775F
:1017270001757801757900F1007C05AD5F1205AC94
:10173700C3ED955F70F5C3E55F9401400AC3E55FAC
:1017470094FF403202175BD166B1C3D1A2C2AF7515
:10175700EF12D19ADCD50579C3E57994035002805D
:10176700C6D19A0578E5771490009F93F808C3E5EA
:101777007898500280AED19AD19A0577C3E57794CD
:101787000A5002809C120EDDB1C3C2AF75EF12D1B1
:011797009AB7
:0319FD0002102DA8
:101A00000E0414FFFFFFFF0304070301015AA501A1
:101A1000FFFFFFFFFF03FFFFFF25D0FAFA04FF01DE
:081A2000007AFF01010003FF41
:101A400023506C6174696E756D31353041232020EF
:101A500023424C48454C4923463331302320202033
:101A60002020202020202020202020202020202076
:101C0000C2AFC2D353D9BF7581C043B20343FF8073
:101C1000752438752503B1C975EF0275E24043F1AB
:101C20000853A4F775D400D2837DFA780379E67C53
:101C300010752200752300901DD67B0675249875BB
:101C400025013083028142208308D8FBD9F9DCF7D3
:101C500081B4308308D8FBD9F9DCF781B4B189E4C9
:101C600093A3C39A6004DDC381B4DBDBB17B600264
:101C7000812B7B08E493FAA3B15CDBF87A30B15C8A
:101C8000752200752300B17BEAFCEBFDC3ED94FEE9
:101C9000400EB17B8A278B28ED30E0048A828B834B
:101CA000B17B7AC270D8C3ED94FE601350CEBD00F4
:101CB00025EC60097520007521FF0200008100A855
:101CC00027A9280809D804D90281D3B17FEA89AAB3
:101CD000F281C50D81A0C3ED94035049EDA2E092BD
:101CE000007AC5C3E5829400E583941C50902000DF
:101CF00010438F02438F0175B7A575B7F1F030001F
:101D00001FA827A9280809438F01538FFDD804D99C
:101D100002A12089AAE275B7A575B7F1F0A3A10DBC
:101D2000538FFC817C7AC1BD030CE493A3FAB140CC
:101D3000DCF8B138817C817EAA22AB23B15CEBFA5E
:101D4000EA6222752608C3E52313F523E52213F57D
:101D50002250066323A0632201D526EAB1C9B1C986
:101D600075260AEAF4200102D283300102C283B14F
:101D7000C9C3134002C201D526EB22B17FEAFB2082
:101D80008302A17F308302A184752608AE24AF258B
:101D9000C3EF13FFEE13FEB1CDB1C9C3EA13308315
:101DA000024480FA30E703632201C3E52313F523DD
:101DB000E52213F52250066323A0632201D526D91C
:101DC000E52265236523F52222AE24AF250E0FDE22
:101DD000FEDFFCD20122424C48656C693437316326
:041DE000F3100601F5
:00000001FF
